:100000000EC029C027C026C0B2C06FC023C022C006
:1000100021C020C01FC01EC01DC01CC01BC0112499
:100020001FBECFE5D1E0DEBFCDBF10E0A0E6B0E05F
:10003000E2E1F4E003C0C89531960D92A436B10711
:10004000D1F710E0A4E6B0E001C01D92AB36B107D5
:10005000E1F7BEC0D5CF1F920F920FB60F921124B9
:100060002F933F934F935F936F937F938F939F93C0
:10007000AF93BF93CF93DF93EF93FF93B29922C0D7
:10008000FAE040ED57E060E070E0E1E0F8BB23E625
:1000900030E0952F842F0197F1F72150304037FF42
:1000A000F8CFE8BBA0EDB7E0C0E0D0E023E630E059
:1000B0008A2F9B2F0197F1F72150304037FFF8CF5F
:1000C000B29BE4CFFF91EF91DF91CF91BF91AF91C0
:1000D0009F918F917F916F915F914F913F912F9160
:1000E0000F900FBE0F901F9018951F920F920FB692
:1000F0000F9211242F933F934F935F936F937F93AE
:100100008F939F93AF93BF93EF93FF9380916A0078
:100110008F5F80936A0080916A0099278F7090703A
:10012000892B41F4EDD08F7380936700E9D08F73F2
:100130008093680080916A0099278F739070892B53
:1001400029F4DED08F77815880936600FF91EF917C
:10015000BF91AF919F918F917F916F915F914F91DF
:100160003F912F910F900FBE0F901F9018951F92E7
:100170000F920FB60F9211248F939F93809164007A
:1001800090916500019790936500809364009F9122
:100190008F910F900FBE0F901F90189588B3847F9A
:1001A00088BB8FE080BDF8940F9305B7006205BF50
:1001B000046805BF0B7F05BF789488950F9180E296
:1001C0009DEF909365008093640083E080BD089567
:1001D000CFE5D1E0DEBFCDBF8BE087BB8FEF88BB23
:1001E00080E886BD16BC80E185BF80E48BBF82E0DD
:1001F00089BF83E083BF89B7846089BF8FE080BFF8
:10020000789480E29DEF9093650080936400C6DF50
:100210008091640090916500892BC9F380916900F9
:100220008F5F8093690090916600809169008917C3
:1002300010F4C09A01C0C098909167008091690045
:10024000891710F4C19A01C0C198909168008091FB
:100250006900891710F4C39ADBCFC398D9CFA0E007
:10026000B0E0E4E3F1E0A5C0D92FC82FE880F98021
:100270000A811B81912F802F7F2D6E2D2DE133EF71
:1002800041E050E067D0A22EB32EC42ED52E912F80
:10029000802F7F2D6E2D2DE133EF41E050E05AD0BD
:1002A00027EA31E440E050E03AD0E62EF72E082F5E
:1002B000192F24E13BE040E050E09D2D8C2D7B2D5B
:1002C0006A2D2DD0E61AF70A080B190BB12FA02FB3
:1002D0009F2D8E2D1E141F041006110624F0815030
:1002E0009040A040B04888839983AA83BB839F77BE
:1002F000A070B070EAE0CDB7DEB777C0B0DF089588
:1003000080E690E0ACDF0895AA27BB2780936000C9
:1003100090936100A0936200B09363000895FF275B
:10032000EE27BB27AA2760FF04C0A20FB31FE41F5C
:10033000F51F220F331F441F551F969587957795FC
:10034000679589F70097760771F79F2F8E2F7B2F80
:100350006A2F0895A1E21A2EAA1BBB1BEA2FFB2FBE
:100360000DC0AA1FBB1FEE1FFF1FA217B307E40794
:10037000F50720F0A21BB30BE40BF50B661F771FEC
:10038000881F991F1A9469F76095709580959095CC
:10039000262F372F482F592F6A2F7B2F8E2F9F2FD5
:1003A00008952F923F924F925F926F927F928F9219
:1003B0009F92AF92BF92CF92DF92EF92FF920F93F4
:1003C0001F93CF93DF93CDB7DEB7CA1BDB0B0FB6FE
:1003D000F894DEBF0FBECDBF09942A8839884888BB
:1003E0005F846E847D848C849B84AA84B984C88451
:1003F000DF80EE80FD800C811B81AA81B981CE0F48
:10040000D11D0FB6F894DEBF0FBECDBFCA2FDB2FB4
:0204100008954D
:0404120001000000E5
:00000001FF
